:0200000067286F
:100008000528CF00030E8301CC000A08CD008A0121
:100018000408CE000B1D2F28AB0F8A1BAA0A383004
:100028002B02031D222801302A02031D22288512D3
:100038000508BE001030BE043E08850035302B028E
:10004800031D2F280C302A02031C2F28AA01AB01FC
:100058003B2085162914A0308B0083014E088400AC
:100068004D088A004C0E8300CF0E4F0E0900223037
:1000780084005B2060302202031C0800A2012130AA
:1000880084005B2060302102031C0800A1010508E0
:10009800BE00EF30BE053E088500203084005B209E
:1000A80024302002031C0800A914A0010800800ABB
:1000B8000008B3000F30B3050A303302031D0800EF
:1000C80006308007080083128501860187018316A0
:1000D800D13081000B30850000308600F030870079
:1000E80004309F00831220308B0080309F0005165B
:1000F800A001A101A2010530A3000130A400013034
:10010800A5000530A600B401A901AA01AB01F03091
:10011800B5008B17AE01AF01B001FE30A8002E303C
:10012800B7000630AA001A30AB008F2199302E0292
:100138000319A5281130AE071130AF071130B007E9
:100148009328A201182100303402031DB52820305D
:10015800B700FE30A80010302002031CA8138F211E
:10016800EF2801303402031DBF282330B700FC30CC
:10017800A8008F21EF2802303402031DCE282F213A
:100188002E30B7003830A80010302F02031CA812F8
:100198008F21EF28EF302207031CAB28EC30220711
:1001A800031CB928DA302207031CAB28D7302207F2
:1001B800031CC328BF302207031CAB28BC3022070E
:1001C800031CB928AA302207031CAB28A730220732
:1001D800031CC328AB28B51BF728B40A0430340223
:1001E8000319B4010929351BFB284C210929351AA3
:1001F80009298B130000AA01AB01A20130302102AA
:10020800031C07294B20A1018B17A91CA628FA213A
:10021800A91001302502031DA62838220130240226
:10022800031DA6284A22A62883169F13831281300D
:100238009F0062221F151F191F291F107D301E07DE
:1002480003182B2978301E02031C2D2908002911B8
:1002580008002915080083169F17831289309F000C
:1002680062221F151F1936291F101E08AC0083169D
:100278001E088312AD000310AC0CAD0C77223008B9
:10028800AF00AF0E3108AF043208B000B00E08005E
:100298008B132330B700C030A8008F21351F582991
:1002A800B51A4F294A224F293030A8008F21351F0F
:1002B8006129B51A5829382258290C30A8008F21ED
:1002C800351F6A29B51A6129FA2161292030B7003A
:1002D800AA01AB01A201F230A8008F21351F7E29A7
:1002E800B51A7129203084005B20243020020318BD
:1002F800A00171298F21351F8B29B51A7E2921303C
:1003080084005B20603021020318A1017E2900309F
:10031800B4008B170800370884000008BB00840A63
:100328000008BC00840A0008BD003B308400A81FF8
:10033800A329800E00088700800E80308600EE21F9
:10034800281FAA290008870040308600EE21840A69
:10035800A81EB429800E00088700800E2030860071
:10036800EE21281EBB290008870010308600EE21E8
:10037800840AA81DC529800E00088700800E083051
:100388008600EE21281DCC2900088700043086004D
:10039800EE21A81CD12902308600EE210708B500FD
:1003A800F030B505F0303502031DDC29B601EA2925
:1003B800B60A013036020319ED293C303602031D16
:1003C800E8293230B600ED29F030B500291C99290A
:1003D800291008005D225D22291986010230B90022
:1003E800672286015D225D225D220800A50A250894
:1003F800A7000F30A7050A302702031D052A06307B
:10040800A50702302402031D1B2A0030230203190A
:10041800152A2608A7000330A7050030270203196C
:10042800182A2830A700302A2930A700302A04309B
:10043800240203192E2A0630240203192E2A093011
:10044800240203192E2A1130240203192E2A3130CE
:10045800A700302A3030A70025082702031C352AB8
:1004680008000130A5000800A40A2408A7000F30DE
:10047800A7050A302702031D432A0630A4071330B4
:100488002402031C08000130A4000800A30AA60ADD
:100498002308A7000F30A7050A302702031D562A94
:1004A8000630A30764302602031C0800A601A30136
:1004B80008006930B900B90B5F2A08001630B90086
:1004C800B90B642A08000030BA00000000000000E0
:1004D800000000000000000000000000BA0B692ABC
:1004E800B90B672A0800BF01C0012C08C1002D08FC
:1004F800C2007F22080032308400C701C801C90148
:100508000A30CA009022460880002E3004020319DF
:100518008F2A8403862A0800C301C401C501C601C5
:100528002030CB000310C20DC10DC00DBF0DC60D8C
:10053800C50DC40DC30D47084302031CB72A031D8C
:10054800B52A48084402031CB72A031DB52A4908DE
:100558004502031CB72A031DB52A4A084602031C94
:10056800B72ABA224214CB0B962A08004A08C602B8
:100578000318C72A0130C5020318C72A0130C4026C
:100588000318C72AC3034908C5020318D02A013033
:10059800C4020318D02AC3034808C4020318D52A82
:0805A800C3034708C302080069
:104200004E00690078006900650054007500620086
:10421000650043006C006F0063006B0020003000FD
:104220002E0036006400200052005500550020008A
:10423000000000000000000000000000000000007E
:10424000000000000000000000000000000000006E
:10425000000000000000000000000000000000005E
:10426000000000000000000000000000000000004E
:10427000000000000000000000000000000000003E
:10428000000000000000000000000000000000002E
:10429000000000000000000000000000000000001E
:1042A000000000000000000000000000000000000E
:1042B00000000000000000000000000000000000FE
:1042C00000000000000000000000000000000000EE
:1042D00000000000000000000000000000000000DE
:1042E00000000000000000000000000000000000CE
:1042F00000000000000000000000000000000000BE
:084000007F007F007F007F00BC
:02400E00323D41
:00000001FF
